:1000000000308A0004280000840183131F30830518
:10001000FF3083169900A230980090308312980028
:1000200083161F149F141F159F1107309C00FF306B
:100030008312A000831681131F149F141F159F1194
:1000400083121F109412A0122008831687008312B7
:1000500020162008831687008312A011200883161B
:100060008700013083129400003083169400010849
:10007000C73908388100831290010030F8009200DF
:1000800000308316920007309C0005086400103091
:10009000F700F70B49281C0883120D1383169D01E6
:1000A00006148312061C582841300C1E552899004E
:0600B000831650286300D6
:02400E00FA3F77
:00000001FF
